:020000040800F2
:10000000080500207D010008870D0008150B000879
:10001000850D0008110B0008210E000800000000EB
:10002000000000000000000000000000AB0D000810
:10003000130B000800000000A90D0008AD0D00081A
:100040009701000897010008970100089701000830
:100050009701000897010008970100089701000820
:100060009701000897010008970100089701000810
:100070009701000897010008970100089701000800
:100080009701000897010008000000009701000890
:100090009701000897010008970100081B0B000852
:1000A00097010008970100089701000897010008D0
:1000B0009701000800000000970100080000000000
:1000C000170B0008000000009701000897010008C6
:1000D0009701000897010008970100080000000040
:1000E00000000000000000009701000897010008D0
:1000F0009701000897010008970100089701000880
:1001000097010008000000000000000097010008AF
:1001100000000000000000000000000000000000DF
:1001200000000000000000000000000000000000CF
:1001300000000000000000000000000000000000BF
:1001400000000000000000000000000000000000AF
:10015000000000000000000097010008970100085F
:100160009701000897010008DFF80CD000F04CFC64
:10017000004800474129000808050020064880473C
:1001800006480047FEE7FEE7FEE7FEE7FEE7FEE77C
:10019000FEE7FEE7FEE7FEE7BD0D00086901000887
:1001A0002DE9F0410024061B254671F1000605DA11
:1001B00001240027D0EB070067EB0101161E73F145
:1001C000000605DA0027D2EB0702012567EB0303DF
:1001D00000F017FA86460E4617469C46AC4204D0FD
:1001E0000025D0EB050E65EB010624B10020D2EB13
:1001F000000760EB030C704631463A466346BDE8A3
:10020000F08140EA01039B0703D009E008C9121FEF
:1002100008C0042AFAD203E011F8013B00F8013BC0
:10022000521EF9D27047D2B201E000F8012B491EEC
:10023000FBD270470022F6E710B513460A46044683
:100240001946FFF7F0FF204610BD30B504460020E8
:10025000034600E05B1C934203D2E05CCD5C401B94
:10026000F8D030BDF0B480EA0102D40F4200B2EB06
:10027000410F02D20246084611464A0042D0C30D41
:10028000DDB2C1F3C752AD1A202D35DAC1F3160124
:1002900041F4000204B15242C5F1200602FA06F10F
:1002A0002A411044B3EBD05F23D0C4B1012DA0EBA1
:1002B000C35009DCF0BC4FF0004202EAC352DBB28B
:1002C00000F5000000F0E7B9400000F1807000EB9D
:1002D000C350A0F1807040EAD170490009E049089C
:1002E00041EAC071A0EBC35000F50000400800EBEC
:1002F000C350F0BC00F0C6B96142012202EB4101DB
:10030000001BF6E7F0BC704781F00041AAE780F0DF
:100310000040A7E780EA010210B502F00043400068
:1003200022D04A001FD0010E01EB1261C0F356002B
:10033000C2F3560240F4000042F40002A0FB022087
:1003400000047F39140400D0401C50EA124001D44C
:100350004000491EC2B20C0604EBD010401C4008FD
:10036000802A02D003E0002010BD20F00100002907
:1003700000DA0020184310BD30B480EA010202F018
:10038000004530F0004221F0004013D090B1C30D81
:10039000D40DC2F31601C0F31600E41A41F40001B3
:1003A00040F400027D34914201D3641C00E0490016
:1003B000002C02DA30BC002070474FF4000000230C
:1003C000914201D3891A034340084FEA4101F7D112
:1003D00051B1914202D14FF0004105E002D24FF0FD
:1003E000010101E06FF0010103EBC450284430BC6F
:1003F00000F048B9420005D0C0F3C75252429142C2
:1004000001DC0020704700EBC15070472DE9FE4F22
:1004100081EA030404F0004421F0004100944FF00D
:10042000000B23F0004350EA01045ED052EA0304BB
:100430005BD0C3F30A54C1F30A552C44A4F2F3343D
:100440000194A0FB0254C1F3130141F48011C3F3E2
:10045000130343F4801301FB024400FB034E840AA0
:10046000970A44EA815447EA8357A4FB0768029538
:100470008D0A05FB07854FEA932C04FB0C542705D6
:10048000029D4FEA065847EA1637B5EB08056EEBB2
:10049000070C870E920E47EA811742EA8312A7FBE8
:1004A0000201B6EB0B0164EB00042B0D43EA0C33A5
:1004B0005E1844EB1C50DA465146E7FB0201C5F3D7
:1004C00013044FEA0B3343EA14534FEA0432019CFE
:1004D00043EA0603A4F10C040294009CCDE900B4A5
:1004E00000F016F903B0BDE8F08F00200146F9E7EF
:1004F000C10F80EAE0700844CA079623002100F08B
:10050000CAB896230022114600F0C5B800F0004298
:1005100020F00040C10DC0F3160040F400007F2918
:1005200001DA00207047962903DCC1F19601C8402A
:1005300001E096398840002AF4D04042704720F00C
:100540000040C10DC0F3160040F400007F2901DA1D
:1005500000207047962903DCC1F19601C84070471E
:1005600096398840704770B5C1F30A5201F00045D2
:100570000024C1F3130140F2FF3341F480119A4289
:1005800001DA002070BD40F233439A42A2F23342B6
:1005900003DC524200F066F800E090402C43F1D0BA
:1005A000404270BD00F0004230F000400AD0C10D62
:1005B00001F56071C0F3160042EA0151C20840071C
:1005C0001143704700200146704701F0004330B4EA
:1005D00021F0004150EA010206D00A0DA2F5607236
:1005E000C1F31301002A02DC30BC00207047440F25
:1005F00044EAC104C100E01830BC00EBC25000F076
:1006000041B82DE9F05F0546002092469B4688469A
:100610000646814640241BE028464146474622467E
:1006200000F020F853465A46C01A914110D31146A3
:100630001846224600F0FAF92D1A67EB01084F46DA
:1006400022460120002100F0F1F917EB00094E418C
:10065000201EA4F10104DFDC484631462A46434609
:10066000BDE8F09F202A04DB203A21FA02F00021A5
:10067000704721FA02F3D040C2F1200291400843B2
:10068000194670470029A8BF7047401C490008BFA1
:1006900020F00100704710B4B0FA80FC00FA0CF0B2
:1006A00050EA010404BF10BC704749B1CCF12004EA
:1006B00021FA04F411FA0CF118BF01212143084377
:1006C000A3EB0C01CB1D4FEA00614FEA102042BFA3
:1006D000002010BC704700EBC35010440029A4BF99
:1006E00010BC7047401C490008BF20F0010010BC3E
:1006F000704710B5141E73F1000408DA401C41F174
:10070000000192185B411A4301D120F0010010BD95
:100710002DE9F04D92469B4611B1B1FA81F202E00B
:10072000B0FA80F22032904600F080F904460F467D
:1007300040EA0A0041EA0B0153465A46084313D0E7
:10074000114653EA010019D0C8F140025046FFF7A4
:1007500089FF05460E4650465946424600F066F966
:10076000084305D0012004E020463946BDE8F08D5D
:100770000020054346EAE0762C4337430A98630598
:10078000E40AA0EB08000022FD0A44EA47540A30BC
:1007900002D500200146E9E7010510196941DDE9AC
:1007A000084500196941BDE8F04DA2E72DE9FE4F6B
:1007B000804681EA0300C00F0C46009021F0004102
:1007C00023F00045B8EB0200A94105D2404621467E
:1007D00090461C460B46024623F00040104347D08B
:1007E000270DC7F30A00C3F30A510290401A019083
:1007F00040286BDAC3F3130040F4801B0098924644
:1008000020B10023D2EB030A63EB0B0B019859468E
:10081000C0F14002504600F009F906460D46504628
:100820005946019A00F011F910EB080061410024CB
:1008300087EA115284EAE7731A4340D0009A62B300
:10084000019A012A4FEA075215DC001B61EB0201F5
:100850004FF0004202EA0752CDE90042001C41F588
:10086000801132462B46FFF753FF03B0BDE8F08FEF
:1008700040462146F9E7001B61EB0201001C41F5EF
:10088000801300185B412018A2F5001747EB030105
:1008900040EAD570B6196D4111E06D084FEA360691
:1008A00045EAC0754FEA0752001B61EB0201001CCC
:1008B00041F5801149084FEA300000195141324694
:1008C0002B4603B0BDE8F04FFFF713BF009801229D
:1008D00040000023D0EB020263EBE0730098214656
:1008E0004FEAE074B8EB000061EB0401E9E783F044
:1008F00000435BE781F0004158E72DE9F04D81EAC4
:10090000030404F0004B21F0004514464FF0000AA8
:1009100023F0004150EA050220D054EA01021DD024
:10092000C5F30A570246C5F31303C1F31300C1F31D
:100930000A5640F4801543F48013A7EB0608101BF9
:10094000D64608F2FD3873EB050002D308F1010822
:1009500001E092185B41B8F1000F03DA0020014674
:10096000BDE8F08D00204FF48011064684460EE06D
:10097000171B73EB050705D3121B63EB0503064337
:100980004CEA010C49084FEA300092185B4150EAEA
:100990000107EDD152EA030012D082EA040083EA93
:1009A0000501084305D0101BAB4106D201220023EC
:1009B00006E000224FF0004302E06FF00102531006
:1009C0001AEB06004CEB085110EB0A0041EB0B014F
:1009D000BDE8F04DFFF78DBE70B521F00043034335
:1009E0000CD0C1F30A550024D5EB040564EB0403D5
:1009F000D617AD1AB34102DB0020014670BD2018A6
:100A000041EB025170BD0000064C074D06E0E06866
:100A100040F0010394E8070098471034AC42F6D345
:100A2000FFF7A6FB0059000820590008202A04DB24
:100A3000203A00FA02F1002070479140C2F12003F1
:100A400020FA03F3194390407047202A06DBCB17A6
:100A5000203A41FA02F043EAE07306E041FA02F379
:100A6000D040C2F1200291400843194670472DE959
:100A7000F04D00231A461B1A8A4103DB0020014671
:100A8000BDE8F08DC1F30A52C1F3130141F48015A2
:100A90004FF0000BD10702D100186D41521E002704
:100AA000044640F2FF11384601EB620A3E4680469A
:100AB000024600204FF48011FFF7D4FDC2197141A6
:100AC000BB1846EB0100B4EB030C75EB000C04D330
:100AD000E41A65EB000517460E46241908F10100DB
:100AE0006D4180463428E3DDF91946EB0600091B09
:100AF000A84103D24FF0FF32134601E00022134613
:100B00001BEB070046EB0A51BDE8F04DFFF7F1BDC6
:100B1000FEE77047FEE700F003B800F059B80000A8
:100B200070B52A4C4FF480652946204601F000FE3E
:100B300018B12946204601F0F2FD4FF40045294640
:100B4000204601F0F5FD18B12946204601F0E7FDE9
:100B50004FF480452946204601F0EAFD18B12946A8
:100B6000204601F0DCFD4FF400652946204601F0E7
:100B7000DFFD18B12946204601F0D1FD4FF4007584
:100B80002946204601F0D4FD18B12946204601F03F
:100B9000C6FD4FF480752946204601F0C9FD18B105
:100BA0002946204601F0BBFD4FF4805529462046DA
:100BB00001F0BEFD18B12946204601F0B0FD2046E7
:100BC000BDE870404FF4E06101F0A1BD0054004069
:100BD0002DE9F05F62480178624FDFF88C81DFF821
:100BE0008CA1634D634C644E4FF000096FF0010B14
:100BF00001290DD0007800283CD195F900004FF074
:100C000001010028304653DB01F092FD28B939E09C
:100C10000121304601F08CFD08B15A464CE002211A
:100C2000304601F085FD00285BD18021304601F07F
:100C30007FFD00281ED095F90000002806DD00BFCA
:100C400098F80010304601F04CFD2DE0207898B166
:100C50004A4A106810F8011B1060304601F041FD4F
:100C60002078401E207000204FF4FA71401C80B2A2
:100C70008842FBD3BDE8F09F304601F0D2FD8AF8F0
:100C8000009066E00221304601F052FD48BB802111
:100C9000304601F04DFD0028ECD095F90000002809
:100CA000CEDC304601F0B8FD2878401E2870E1E720
:100CB00001F03EFD30B1012239783046BDE8F05FE9
:100CC00001F052BD0221304601F032FD78B12078AA
:100CD000012802D02078022803D10021304601F0FB
:100CE00075FC3046BDE8F05F022101F018BD4021DF
:100CF000304601F01DFD0028BCD020780028B9D076
:100D00002078032809D10421304601F011FD002884
:100D1000F9D00021304601F059FC304601F0DEFCEC
:100D200017490246086800F8012B08602078401E29
:100D30002070207800289DD1304601F072FD8AF89D
:100D400000900121304601F041FC0121304601F0C4
:100D500047FC3046BDE8F05F4FF4E06101F0D7BCDE
:100D60002D0000202F0000202E0000202C0000204D
:100D700031000020300000200054004034000020EA
:100D800038000020FEE770470907090E002806DA40
:100D900000F00F0000F1E02080F8141D704700F112
:100DA000E02080F8001470477047704710B503F0DA
:100DB000CFFDBDE8104000F019BC000014480168E8
:100DC00041F00101016001688907FCD54168114AC1
:100DD000114041604168104A11404160416821F46E
:100DE0004001416001680D4A11400160C16A21F073
:100DF0000F01C162016B40F2431291430163416BE9
:100E000021F0010141630021816003F059BD000020
:100E1000001002400C00FF08FFFFC277FFFFF2FE48
:100E2000FEE7490050EAC12018BF04204A0D18BF50
:100E300040F0010040F2FF72B2EB515F08BF40F09A
:100E40000200012808BF052070472DE9F0414F1E20
:100E500000EBC7010446D1E9000115461E4637F0F4
:100E600006020DD02A463346FFF7D0FA7F1E04EB68
:100E7000C703D3E90023FFF799FC37F00602F1D14D
:100E8000022F25D0042F13D0062F18BFBDE8F08104
:100E90002A463346FFF7BAFAD4E90A23FFF786FC5D
:100EA0002A463346FFF7B2FAD4E90823FFF77EFC5F
:100EB0002A463346FFF7AAFAD4E90623FFF776FC61
:100EC0002A463346FFF7A2FAD4E90423FFF76EFC63
:100ED0002A463346FFF79AFAD4E90223FFF766FC65
:100EE0002A463346FFF792FAD4E90023BDE8F041E1
:100EF000FFF75CBC0122FFF76FBDFFF757BC002274
:100F0000134610461146FFF7F8BC0000024A0020C5
:100F10001107FFF761BD000001FDFFFF02E008C8F7
:100F2000121F08C1002AFAD170477047002001E063
:100F300001C1121F002AFBD170470000014908605F
:100F4000704700006C0000202DE9FE4F07460E465A
:100F50000025684600F094FF00246FF00F0AE84671
:100F60004FF0010957F8240056F82410401A00D514
:100F70004042FFF7BDFA5146FFF73CFA58F82410FB
:100F800011F0FF4F0BD0FFF7F7F94FF07E51FFF74D
:100F9000BBF90A4920F00040884205DC07E0084917
:100FA00008440849884202D309FA04F00543641C46
:100FB000032CD7DB2846BDE8FE8F0000295C0F3EDE
:100FC000666666C19A99D9002DE9F04D8D4F21F0E2
:100FD000004A86B005460C46BA452ADBAAEB070054
:100FE00028430AD08848824501DC1AD1CDB106B029
:100FF0002846BDE8F04DFFF77DBF844A844B284664
:10100000FFF704FA07460E46824A834B28462146DC
:10101000FFF7FCF906B03A463346BDE8F04DFFF75E
:10102000C5BB0120FFF78AFF06B0BDE8F04DFFF712
:1010300066BF7A48824542DABAF1795F0BDA284610
:10104000FFF7EFFE042808BFFFF760FF284606B051
:101050002146BDE8F08D2A460B461046FFF7D6F92B
:10106000834602466E480E460B4606217844FFF73B
:10107000ECFE5A463346FFF7C9F9804669488A466E
:101080005A46334604217844FFF7DFFE5A4633467A
:10109000FFF7BCF900223B46FFF788FB02460B46F0
:1010A00040465146FFF729FC2A462346FFF7AEF992
:1010B00006B02A462346BDE8F04DFFF777BB284629
:1010C00024F0004100223D463B46FFF713FC4FF061
:1010D000FF32FFF781FC0646024653480F460B4697
:1010E00006217844FFF7B1FE32463B46FFF78EF902
:1010F000CDE900014D4832463B4604217844FFF7D4
:10110000A4FE32463B46FFF781F900222B46FFF74B
:101110004DFB834602913046394603F0ABFB8046D7
:1011200043480D46504517DCDDE900015A46029B55
:10113000FFF7E3FB42462B46FFF768F942462B4692
:10114000FFF734FB0122FFF747FC304A304BFFF733
:10115000CEFB304A304B4CE04FF0000A52460B4673
:101160004046FFF723FBCDE9031052462B461046BD
:101170001946FFF74BF932463B46FFF7BBFBDDE96B
:101180000332FFF7BAFB06460F46DDE900015A4677
:10119000029BFFF7B2FB834600910122304639469D
:1011A000FFF71AFC194A1A4BFFF7A4FB06460F4635
:1011B000012240462946FFF70FFC5A46009BFFF7E5
:1011C00025F932463B46FFF792FB06460F460122C1
:1011D00050462946FFF700FC0E4DDFF858802A469E
:1011E0004346FFF787FB32463B46FFF783FB2A4621
:1011F0004346FFF77FFB002CD8BF81F0004106B0CB
:10120000BDE8F08D0000F03F0000F07F075C143374
:1012100026A6913C182D4454FB21F93F0000E03FE5
:10122000A0470000B64700002A47000040470000E2
:101230003333EF3FFB21E93F2DE9F84F04460D46DC
:1012400021F0004000917349814211DC72498842CB
:1012500001DC06D12CB120462946BDE8F84FFFF746
:1012600049BE6E48002DCCBF6D496E49BDE8F88F70
:101270006D49814211DD6D498142D8BF4FF0FF3683
:101280006DDD20462946FFF7CCFD042808BFFFF797
:101290003DFE20462946BDE8F88F6549654F25F09B
:1012A0000045814233DD6449814219DD0026324622
:1012B0004FF0804320462946FFF778FA80468A4659
:1012C000012220462946FFF787FB00223B46FFF715
:1012D0000EFB42465346FFF710FB04460D463EE028
:1012E00001260022BA463B4620462946FFF75EFA11
:1012F00080460F460022534620462946FFF7F7FA5C
:1013000042463B46FFF7F9FA04460D4627E04B49B3
:1013100081421BDDDFF828A1022600225346204629
:101320002946FFF773F800223B46FFF73FFA804655
:101330000F460022534620462946FFF7D8FA424678
:101340003B46FFF7DAFA04460D4608E0032622463C
:101350002B4600203B49FFF7D0FA04460D462246B3
:101360002B4610461946FFF751F88B468246024637
:101370000B46FFF74BF807460246334888460B46B4
:1013800006217844FFF761FD52465B46FFF73EF8C1
:1013900082462E488B463A46434605217844FFF75D
:1013A00054FD3A464346FFF731F802460B46002EFD
:1013B000504659460CDAFFF7F9F922462B46FFF75B
:1013C00025F801B022462B46BDE8F04FFFF792BA50
:1013D000FFF7ECF922462B46FFF718F81C4A7A442F
:1013E00002EBC603D3E90023FFF781FA22462B461E
:1013F000FFF77DFA174A7A4402EBC603D3E90023CC
:10140000FFF778FA009A002AB8BF81F00041BDE8E2
:10141000F88F0000000010440000F07F182D4454A5
:10142000FB21F93FFB21F9BF0000DC3F0000203E1B
:101430000000F33F0000F03F0000E63F0080034063
:101440000000F83F0000F0BF4245000000450000EA
:101450009E440000664400002DE9F04D9446CCF116
:10146000000423F000464CEA0404524F46EAD474C8
:101470009A46884621F00042BC4206D8454240EADE
:10148000050442EAD474BC4204D9BDE8F04D62467A
:10149000FFF733BDAAF14055A5F17F6555EA0C046D
:1014A0000BD0022404EAAA74434DDFF810E144EAA9
:1014B000D87452EA000B04D00CE0BDE8F04DFFF701
:1014C000BBBE002C14BF012CBDE8F08D022C30D027
:1014D000032C32D056EA0C0B0AD0BE4220D1BA42BD
:1014E00009D126F0804622F080423346114617E0AB
:1014F00000291ADB25E0DFF8C8B0FB44002C04BF4C
:10150000DBE90001BDE8F08D012C02BFDBE9000141
:1015100081F00041BDE8F08D022C0AD0032C0CD0E4
:10152000BA4212D1B8F1000F0BDA23482549BDE8C1
:10153000F08D28462449BDE8F08D28467146BDE867
:10154000F08D1D482149BDE8F08D921B12153C2AF3
:10155000C4BF19481D490EDCBAF1000FBEBF12F11D
:101560003C0F0020014606DB6246FFF7C6F921F07A
:101570000041FFF761FE002C08BFBDE8F08D012C93
:1015800004BF81F00041BDE8F08D114A114B022CDF
:1015900007D0FFF7ACF92A46BDE8F04D0A4BFFF73C
:1015A000A6B9FFF7A4F92A46BDE8F04D064BFFF7B0
:1015B000A1B900000000F07F182D4454FB2109C0A0
:1015C000FA430000FB21F9BFFB210940FB21F93F51
:1015D000075C143326A6A13C70470000024948600E
:1015E00048680028FCD17047240000200348416867
:1015F000002902D04168491E416070472400002044
:1016000000EB8000810003480844816821F001015B
:10161000816070470000024000EB800081000348B9
:101620000844816841F00101816070470000024078
:1016300000EB8000810003480844816821F020010C
:10164000816070470000024000EB80008100034889
:101650000844816841F02001816070470000024029
:101660000A4B00EB800103EB81018A6822F0010242
:101670008A6000228A60CA600A614A6159688200F1
:101680000F20904001435960704700000000024065
:10169000044A1268800081400A4201D0012070474C
:1016A00000207047000002402DE9F0430DF11C08B6
:1016B00000EB800098E8E0024FEA80081548DDE979
:1016C0000BC4404401614561C0F80CC081683243DD
:1016D00021F47C510C4322438260816883B121F064
:1016E00040018160816877B121F08001816081686B
:1016F000B9F1000F0AD041F010018160BDE8F0831C
:1017000041F04001EDE741F08001EFE721F01001E9
:10171000F3E700000000024000EB80008100034876
:101720000844816821F480418160704700000240D4
:1017300008B560B120208DF8000028208DF8010048
:1017400030208DF8020038208DF8030004E0A32239
:1017500004216846FEF767FD6A46042140F69E2094
:1017600002F002FF02F00EFB08BD00003EB5044689
:1017700002208DF80000CA208DF80100E3208DF8CA
:10178000020009208DF803006A460421682002F057
:10179000EBFEA3208DF80000610609D5C0218DF86D
:1017A0000110C8218DF80210C2218DF8031005E048
:1017B0008DF801008DF802008DF8030014F4C07F4D
:1017C00009D0C4218DF80410CC218DF80510C62154
:1017D0008DF8061005E08DF804008DF805008DF8F1
:1017E00006008DF808008DF807008DF809006A469C
:1017F0000A2140F6A72002F0B7FEA0074FF0D80557
:1018000003D020208DF8000001E08DF800506A46DA
:10181000012140F6B62002F0A7FEA00601D5012066
:1018200000E0002000F08EF814F4C07F1ED0E00528
:101830000AD5B2208DF800008B208DF80100B6206B
:101840008DF802009B2009E0B0208DF80000802078
:101850008DF80100B4208DF8020090208DF803006F
:101860006A46042140F6A22002F07EFEE1074FF412
:101870000B6022D0F8218DF800106A46012102F099
:1018800073FEFA21072000F047FA072000F013FA50
:10189000012000F030FA642000F0D2FA4FF4FA7020
:1018A00000F0DEFAC821254800F0CDF9282000F02C
:1018B000E2F90A2000F0EFF905E08DF800506A46E1
:1018C000012102F051FEA00703D5D9208DF80000B8
:1018D00001E08DF800506A46012140F23D7002F0AF
:1018E00043FE600701D5012000E0002000F048F829
:1018F000E00601D5012000E00020FFF719FF104DA0
:1019000044F00800688102F03DFA0020A8736006E8
:1019100001D50620A87314F4C07F02D0A87B801DD7
:10192000A87314F0140F02D0A87B1030A873A0077E
:1019300002D0A87B001DA87300203EBD09E3CA02A7
:10194000F40000200EB54FF4976310B106A107C94B
:1019500001E008A207CA8DE807006A460921184677
:1019600002F002FE0EBD0000B8AAB38DB4980D358A
:101970005D000000B8AAAAAAB088C3C5C7000000CD
:1019800008B560B1C0208DF80000C2208DF80100BC
:10199000C4208DF80200C6208DF8030004E08B22DD
:1019A00004216846FEF73FFC6A46042140F6982071
:1019B00002F0DAFD02F0E6F908BD0000024989896B
:1019C0000180002070470000F4000020C8234FF47D
:1019D0008062024940F6F63001F0E4BF144C000882
:1019E0002DE9FF4F89B01746DDE9165200244C4E11
:1019F000884681462C80A246B07B694602F030F9C9
:101A00004FF0FF3B18B158460DB0BDE8F08F70891C
:101A100010F0140F3CD0009909BA21F0FF039DF893
:101A200003100B433B6001991B1409BA21F0FF021C
:101A30009DF807105B430A437A6002999DF80B40BA
:101A400009BA21F0FF012143B960039C091424BAAB
:101A500024F0FF0C9DF80F4012144CEA040CC7F858
:101A60000CC04FEA2C47494302FB023207FB071127
:101A700011441024A1F17061B1F1007F04D902F08A
:101A800081F9A5F800A0BEE7298841F4807129807A
:101A90004206694611D50A19A41D13885BBAA8F835
:101AA000003053885BBAA8F80230928852BAA8F87E
:101AB00004202A8842F008022A8010F4C07F11D046
:101AC0000A19A41D13885BBAA9F8003053885BBAC1
:101AD000A9F80230928852BAA9F804202A8842F064
:101AE00070022A80800716D00C44E07800F0C00510
:101AF00000F03F016078C00706D0C80801F0070178
:101B00003268491C02B190476078000703D57168BC
:101B100009B1A80988470C9800F092FB002073E7F0
:101B2000F40000200149486000207047F4000020C4
:101B30000149086000207047F400002030B50446D9
:101B400013A285B007CA8DE807004FF0FF35C82CF7
:101B500016D8C820B0FBF4F1491E080A8DF80C0015
:101B60008DF80D1003AA022140F2162002F0FCFCB1
:101B700030B96A460C2140F6C12002F0F5FC10B1E4
:101B8000284605B030BD054884810020F9E70000F3
:101B9000FEF2ABC4AAF1DFDFBBAFDFDFF400002051
:101BA00000B50EA187B00EC98DE80E000EA10DF193
:101BB0000C0C0EC98CE80E0040F68223012807D0D9
:101BC000022803D04FF0FF3007B000BD6A4600E0A6
:101BD00003AA0B21184602F0C7FCF5E7D8B1B9F308
:101BE0008BA391B609B4D900DAB1B9F38BA391B63E
:101BF000DAB4DA0008B5010E8DF80010010C8DF88A
:101C00000110010A8DF802108DF803006A460421C4
:101C10004FF4587002F0A8FC08BD1421B0FBF1F09D
:101C200008B5010E8DF80010010C8DF80110010AA5
:101C30008DF802108DF803006A4604214FF471708C
:101C400002F092FC08BD4FF47A7290FBF2F008B5F6
:101C50004843010E8DF80010010C8DF80110010AA7
:101C60008DF802108DF803006A4604214FF4AE701F
:101C700002F07AFC08BD0521B0FBF1F008B5010ABD
:101C80008DF800108DF801006A4602214FF4AD7006
:101C900002F06AFC08BD0521B0FBF1F008B5010AAD
:101CA0008DF800108DF801006A4602214FF4AC70E7
:101CB00002F05AFC08BD08B500218DF80010C107DC
:101CC00002D030218DF80010810705D59DF8001055
:101CD00041F00C018DF80010400705D59DF800007B
:101CE00040F003008DF800006A4601214FF4A47013
:101CF00002F03AFC08BD08B560B1042800D9042000
:101D0000401E8DF800006A46012140F24F1002F09B
:101D10002BFC08BD0120F3E72DE9FC4105464007F7
:101D20004FF0FF367CD0B1F5C86F79D80846FEF782
:101D3000E8FB3E49FEF720FB074601A801F0D8F872
:101D40009DF80400022806D004280DD008282ED0C3
:101D5000102865D134E00E213846FEF74BFBFEF724
:101D6000EEFB84B2324907E00D213846FEF742FB14
:101D7000FEF7E5FB2F4984B23846FEF7CBFAFEF7B3
:101D8000DEFB210A8DF8001080B28DF80140010AB7
:101D90008DF802108DF80300E8076C4620D022462B
:101DA00002214FF4EA7002F0DFFBC8BB11E00C2106
:101DB0003846FEF71FFBFEF7C2FB84B21E49DBE785
:101DC0000B213846FEF716FBFEF7B9FB84B21B4920
:101DD000D2E7A21C02214FF4927002F0C5FBF8B9C1
:101DE000A8070DD56A4602214FF4EC7002F0BCFB47
:101DF000B0B9A21C02214FF4947002F0B5FB78B97F
:101E0000680710D56A4602214FF4EE7002F0ACFB71
:101E100030B9A21C02214FF4967002F0A5FB10B15C
:101E20003046BDE8FC810020FBE70000000048438D
:101E3000000040460000C045000040450000C0448E
:101E40000521B0FBF1F008B5010A8DF800108DF8FE
:101E500001006A4602214FF4EF7002F085FB08BDD5
:101E60000521B0FBF1F008B5010A8DF800108DF8DE
:101E700001006A4602214FF4ED7002F075FB08BDC7
:101E80002DE9FE430646264801AB042240680D2199
:101E9000007800F091FC10B10720BDE8FE839DF8AA
:101EA00004101C2000EAD1029DF80710DFF874909E
:101EB000C1F301131A438DF800209DF80520C1F3EA
:101EC000810300EAD2021A438DF801209DF8062012
:101ED00001F0030100EAD20008430024124F8DF8FC
:101EE0000200A0466D46285D10B146F824900AE035
:101EF00046F824800DE000BF56F824003946FEF76E
:101F000009FA46F82400285D401E10F0FF0028550D
:101F1000F2D1641CE4B2032CE5D30020BDE700003D
:101F2000400000207B14AE3E1D5A843F2DE9FE4F39
:101F300005460120C14E8DF800004FF000088DF8D5
:101F4000018030680C461746417D70686B4602225E
:101F5000007800F06BFC4FF0FF3A00287AD1C820DF
:101F6000FFF73CFB8DF8008030686B460122417C16
:101F70007068007800F05AFC0028EFD130686B469A
:101F8000012241797068007800F050FC0028E5D10A
:101F900030686B460122417D7068007800F046FC95
:101FA0000028DBD130686B460122817E70680078A2
:101FB00000F03CFC0028D1D130686B460122017949
:101FC0007068007800F032FC0028C7D14FF00C098F
:101FD0008DF8009030686B460122017970680078B6
:101FE00000F024FC002835D10F20FFF7F7FAB06A83
:101FF0006B460122407A8DF8000030688178706865
:10200000007800F013FC002824D1B06A6B4601224E
:10201000007A8DF80000306841787068007800F030
:1020200005FC002873D1B06A807A0FB140F0E0005F
:102030008DF8000030686B46012281797068007865
:1020400000F0F4FB002862D12FB1B06AC07A40F0F2
:10205000E00001E04AE018208DF8000030686B468F
:102060000122C1797068007800F0E0FBF0BB17B185
:10207000C820FFF7B3FA40208DF8000030686B46A7
:10208000012201797068007800F0D0FB70BB7820E5
:102090008DF8000030686B46012241797068007845
:1020A00000F0C4FB10BB3220FFF798FA8DF80080D7
:1020B000306847466B46417970680122007800F02D
:1020C000B5FB98B931687068B046097B00786B46FB
:1020D000022200F071FB48B9BDF80000AF6040BAC1
:1020E000B0FBF9F06F60C6B22F6000E00FE0A760B0
:1020F00067602760002739E0D8F80010D8F804009E
:102100006B46497B00780C2200F056FB10B150461C
:10211000BDE8FE8FBDF80000236840BA02B2BDF8EA
:102120000200BDF804101A44226040BA626800B28E
:102130001044606049BAA06809B20844A060BDF8C4
:1021400006002B6840BA02B2BDF808001A4440BA33
:1021500001B2BDF80A002A606A6840BA1144696099
:10216000A96800B208447F1CFFB2A860B742C3D37D
:1021700028688322C117090441EA104100040023A2
:10218000FEF70EF832460023FEF70AF8286068686A
:102190008322C117090441EA104100040023FDF71E
:1021A000FFFF32460023FDF7FBFF6860A86883222B
:1021B000C117090441EA104100040023FDF7F0FFB4
:1021C00032460023FDF7ECFFA86020684FF400655D
:1021D000C117090441EA104100042A460023FDF713
:1021E000DFFF32460023FDF7DBFF206060682A46F0
:1021F000C117090441EA104100040023FDF7D0FF94
:1022000032460023FDF7CCFF6060A0682A46C11764
:10221000090441EA104100040023FDF7C1FF3246E2
:102220000023FDF7BDFFA060002802DDA0F580308F
:1022300001E000F58030A060002069E74000002048
:10224000014909680160704724000020F0B5036A65
:10225000446A002501260F2706FA05FC1CEA020F36
:1022600009D04FEA850C07FA0CFE23EA0E0301FAA7
:102270000CFE4EEA03036D1CADB2082DECD308250D
:1022800006FA05FC1CEA020F0BD04FEA850CACF1F4
:10229000200C07FA0CFE24EA0E0401FA0CFE4EEAAA
:1022A00004046D1CADB2102DEAD303624462F0BD8C
:1022B00081627047816170472DE9F04740F2115605
:1022C000304602F081FA771C384602F07DFA01238D
:1022D0004FF0904800221946404600F0CAF8DFF857
:1022E00080914FF40074234600220121484600F0FB
:1022F000C0F865102B4600220121484600F0B9F8CD
:10230000202300220121484600F0B3F810230022C8
:102310000121484600F0ADF8012303220021404688
:1023200000F0CAF8234603220021484600F0C4F812
:102330002B4603220021484600F0BEF8202303224A
:102340000021484600F0B8F8102303220021484637
:1023500000F0B2F801214046FFF7AAFF21464846A7
:10236000FFF7A6FF29464846FFF7A2FF202148466F
:10237000FFF79EFF10214846FFF79AFF304602F014
:1023800023FAB41C204602F01FFA00221023114643
:10239000404600F06EF8AB01324D0022114628464F
:1023A00000F067F8384602F00FFA40F2157002F0BC
:1023B0000BFA402201214846FFF748FF8022012105
:1023C0004846FFF743FF402301220221484600F020
:1023D00050F8402303220121484600F06DF8802385
:1023E00001220221484600F044F880230322012103
:1023F000484600F061F8304602F0E6F9384602F04F
:10240000E3F9204602F0E0F900224FF400431146C0
:10241000284600F02EF8022300220121404600F059
:1024200028F84FF48064234600220121484600F03A
:1024300020F8022303220021404600F03DF8234605
:1024400003220021484600F037F802214046FFF7FA
:102450002FFF21464846BDE8F047FFF729BF00009F
:1024600000040048000800480069084000D001202E
:1024700070472DE9F047894601689246C2680024FA
:1024800001274FF0030C07FA04F51D420BD066003C
:102490000CFA06F5A943AA4309FA06F80AFA06F562
:1024A00048EA01012A43641CA4B2102CEBD301605A
:1024B000C260BDE8F0870000F0B50129416819D07D
:1024C000994341608168002401274FF0030C00BF4D
:1024D00007FA04F61E4207D066000CFA06F521EA58
:1024E000050502FA06F12943641CA4B2102CEFD3AF
:1024F0008160F0BD1943E4E72DE9F84F81462E488D
:102500008846002540686B46032200780D2100F0C4
:1025100053F910B10720BDE8F88F9DF800000024A2
:1025200000F01F008DF800009DF801006FF00F0B08
:1025300000F01F008DF801009DF802006E4600F0CB
:102540001F008DF802004FF0010A00BF59F8241057
:1025500058F82400081A00D54042FDF7C9FF594633
:10256000FDF748FF0746305DC0B1144802E014494A
:10257000FDF7D0FE315D491E11F0FF013155F6D156
:1025800001463846FDF7F8FE4FF07E51FDF7BCFEE0
:102590000C4920F00040884205DC07E00A48384436
:1025A000B0F1D97F02D90AFA04F00543641C032C68
:1025B000CCDB2846AFE70000400000200000C84107
:1025C00054E3853F295C0F3E0000E0BE012901680D
:1025D00003D021F480610160704741F48061FAE723
:1025E0000029016803D021F400610160704741F4C3
:1025F0000061FAE770B5044616460D46022002F067
:102600002DF8254BB0FBF3F13F2900D33F21626841
:1026100022F03F020A436260204A954210D8B0FB84
:10262000F3F1491C3F2900D33F2121626900B0FB2F
:10263000F1F0042800D20420E169C0F30B0028E087
:10264000174A954227D84FF4967251434FF47A7245
:10265000B1FBF2F1491C216266B105EBC50101EB4A
:102660000511B0FBF1F0E16941F48041E161010540
:1026700008D009E005EB4501B0FBF1F0E16921F478
:102680008041F3E740F00100E16941F40041E1617C
:10269000E1690143E16170BD40420F00A086010085
:1026A000801A060010B50C4C4FF4804209492046B0
:1026B000FFF7A0FF002224231146204600F05DF81A
:1026C000204600F010F82046BDE810400121FFF739
:1026D0007DBF0000801A0600005400400069C0B2AF
:1026E000704701617047016841F001010160704766
:1026F000024601F00043002089B2B3F1004F04D03C
:1027000052690A4200D0012070479269F9E7426895
:102710008A434260704742680A4342607047022918
:1027200003D042698A4342617047416980697047BA
:1027300010B5426802F40073426811F0FF0F02F412
:10274000807206D02BB1CA0607D1426802F48062BB
:1027500002E011F47F4F05D022B14069084000D05B
:10276000012010BD002010BD921C03D041F00101DA
:102770000161704721F00101FAE710B5046824F007
:1027800002040C4304601A43826010BD10B54FF47C
:10279000C06001F059FF03220021172001F00EFF55
:1027A00002220021BDE81040202001F007BF13469F
:1027B000012200F001B8000070B5144C00256570CE
:1027C000FF2525704000E070A170E36022710120B8
:1027D00060710F4D4FF4E0612846FFF79CFF2079B0
:1027E000022803D100212846FFF7FAFE094E2846A9
:1027F0003146FFF77DFF0028F9D1284600F00CF89C
:1028000020790028FCD194F9000070BD2C00002034
:102810000054004002000080016841F480710160B2
:102820007047016841F400710160704770B5104C49
:1028300001256570FF2626704000E070A170A3603E
:10284000227165710B4D4FF4E0612846FFF763FF7D
:10285000094E28463146FFF74BFF0028F9D128469C
:10286000FFF7DAFF20790028FCD194F9000070BD51
:102870002C00002000540040020000802DE9F047A9
:102880002E4D814600274FF090444FF480784FF44E
:10289000007601212046FFF70DFD41462846FFF74F
:1028A00007FD4846FEF79AFE31462846FFF702FD2F
:1028B00001212046FFF7FCFC4846FEF78FFE41460B
:1028C0002846FFF7F7FC31462846FFF7F1FC48465B
:1028D000FEF784FE7F1C062FDBDB0027012120464C
:1028E000FFF7E8FC31462846FFF7E4FC414628465E
:1028F000FFF7E0FC20212846FFF7DCFC10212846EA
:10290000FFF7D8FC4846FEF769FE01212046FFF795
:10291000CFFC31462846FFF7CBFC41462846FFF75F
:10292000C7FC20212846FFF7C3FC10212846FFF7EB
:10293000BFFC7F1C022FD1DBBDE8F08700040048FC
:1029400001F0E6FFFFF7B8FC8C4C4FF4164120462F
:1029500002F09CF8FFF7A6FEFFF718FF0C2288494B
:10296000204602F02FF8864914222031204601F03B
:10297000F7FF6420FFF782FF00F01CFA814C00266D
:1029800000B16670682000F0FFFBDFF8F4B10127AA
:1029900032254AF6AA290BF1200B4FF0904A01206C
:1029A000FEF71CFE6078012808D001214FEA0A00DA
:1029B000FFF780FC6078012804D005E04FF4007137
:1029C0007148F5E700F0B2FAA068B0FBF5F105FB3D
:1029D000110020B96078012801D101F08FF8102191
:1029E0005046FFF741FD58B1A77020216648FFF718
:1029F00061FC66A0FEF7F0FD3220FEF7EFFD04E07B
:102A0000A67020216048FFF753FC4FF480416548D1
:102A1000FFF72AFD58B1E77010215B48FFF74AFC29
:102A200061A0FEF7D9FD3220FEF7D8FD04E0E67084
:102A300010215548FFF73CFCA168B1FBF5F005FB00
:102A4000101080BB02210320FEF722FE01282AD1AC
:102A50004B495B4ADFF828C1A1F80090938B4B806B
:102A6000D18BACF80410128CACF8062094F802C09C
:102A700094F8038048464CEA480CDFF8048158403B
:102A8000514048404146A8F808C080EA0C004881FF
:102A90000320FEF7B5FD4B480C21816441460165DA
:102AA0000320FEF7B9FDBBF80020BBF80230BBF8ED
:102AB00006C082EA0301BBF8043083EA0C035940E4
:102AC000BBF808305940BBF80A305940BBF80C300D
:102AD0005940BBF80E305940BBF8103059401FFA2E
:102AE00081FC4A451BD1BBF91200D846604516D17E
:102AF000207838B1B4F90410481EA08000292FDCDA
:102B0000267032E01E4914222031A1F11400FDF795
:102B100078FB4FF6FF70A8F80000A68025E0B4F916
:102B20000410481CA0804FF49670814201DB27708E
:102B3000A080A068B0FBF5F105FB110070B94A4513
:102B40000CD0A2F57F40FF3808D00420FEF758FDD6
:102B50000B4914222031094801F002FF207820B1EE
:102B600001215046FFF7A6FB03E001215046FFF785
:102B70009FFBA068401CA06011E7000000440040DB
:102B80007000002004000020000400482D2D205378
:102B9000454E534F52203120416374697665202D94
:102BA0002D0A0000000800482D2D2053454E534F9C
:102BB00052203220416374697665202D2D0A000071
:102BC000D00000200000024040B1012808D00228B7
:102BD00008D0032808D105A0FEF7FEBC08A0FBE73B
:102BE00004A0F9E709A0F7E7704700005265766591
:102BF000727365204C616E6473636170650A0000D6
:102C0000506F7274726169740A00000052657665D3
:102C100072736520506F7274726169740A000000EB
:102C20002DE9FC5F5F4CE068FDF762FC6FF01D056D
:102C30002946FDF7DFFB00902069FDF759FC294686
:102C4000FDF7D8FB81466069FDF752FC2946FDF788
:102C5000D1FB8046A069FDF74BFC2946FDF7CAFB76
:102C6000064641460846FDF755FB05464946019094
:102C70000846FDF74FFB2946FDF7F4FA0121FDF761
:102C8000B9FB4FF07E51FDF742FBFDF78BFC074689
:102C90000D4631464046FDF73DFB824649460098C9
:102CA000FDF738FB5146FDF7DDFA0121FDF7A2FBE8
:102CB000FDF778FC3A462B46FEF7CEFBFDF785FC88
:102CC000834649463046FDF725FB054641460098B8
:102CD000FDF720FB2946FDF717FB0121FDF78AFBD5
:102CE000FDF760FCFEF770F9FDF76FFC8246314698
:102CF0000846FDF70FFB01460198FDF7B3FA0121E5
:102D0000FDF778FB4FF07E51FDF701FBFDF74AFC24
:102D100007460D4641464846FDF7FCFA80463146D7
:102D20000098FDF7F7FA4146FDF79CFA0121FDF7FF
:102D300061FBFDF737FC3A462B46FEF78DFBFDF7AE
:102D400044FC05465846FDF72DFC174E174F3246FA
:102D50003B46FDF75BFBDFF8588000224346FDF75A
:102D600055FBFDF700FCA0835046FDF71BFC3246E7
:102D70003B46FDF74BFB00224346FDF747FBFDF7C3
:102D8000F2FBE0832846FDF70DFC32463B46FDF79B
:102D90003DFB00224346FDF739FBFDF7E4FB2084B1
:102DA000BDE8FC9FD0000020F8C1631ADCA54C40B0
:102DB0000000594070B51EA0FEF70EFC00F094FD17
:102DC0004FF0FF3508B121A017E0782001F0BEFADE
:102DD000782000F063F8142001F078FA1F4C0320EB
:102DE00000216070A1706161E1601DA02161FEF7AA
:102DF000F3FBFEF7EBFD20B11EA0FEF7EDFB28462E
:102E000070BD2148FEF794FE2048FEF78BFEF320AC
:102E10002083FEF7ABFC1420FEF790FE012001F0AA
:102E20007BF90120A0701AA0FEF7D6FB002070BD30
:102E30002D2D20436F6E6669677572696E67204D30
:102E40005055363035302E2E2E2000004641494C4C
:102E500020284D5055292E0A00000000A400002013
:102E60002077726974696E6720444D502E2E2E2093
:102E700000000000204641494C2028444D502920A4
:102E80002D2D0D0A000000000D450008C92B00087B
:102E9000204F4B202D2D0D0A000000002DE9F041A0
:102EA000124C20F00101002594F8240010B10020FC
:102EB000BDE8F081A07A4FF0FF3668B10840277C6A
:102EC0002074884200D0354641B1012001F0A6FCB3
:102ED00000F058FF38B127743046E9E7207D00B193
:102EE000012001F09BFC2846E2E7000040000020A2
:102EF0000D494A7A42B1012A08D0022A0FD0032A8A
:102F00000FD04FF0FF307047022200E00422027021
:102F1000C97C11B11106C90D01700020704708224B
:102F2000F5E71022F3E70000400000202DE9F04112
:102F300052488CB000260168406809AAC97C007814
:102F4000FFF735FC9DF824004D4D80074FF0010838
:102F500001D085F8048008A8FFF772F9296908985C
:102F6000814203D200F5FA70012628612879444C89
:102F700000272C34F0B3A878E0B30AA906A8CDE95D
:102F8000000107ABA4F1100204A902A8FEF728FD76
:102F90009DF8280000B92F71BDF8180010F0700FCF
:102FA00015D0BDF808002080BDF80A006080BDF88B
:102FB0000C00A0805EB1314807A9001F00F0A6F800
:102FC0002E486421001F0068484300146084BDF946
:102FD0001800010708D5BDF81010E180BDF81210E7
:102FE0002181BDF814106181C0050DD524481C3025
:102FF000016800E00BE0E160416821618168616186
:10300000C068A061FFF70CFE0CB0BDE8F081287924
:103010000028F9D02F710AA8009005AB07AA03A9D0
:1030200001A800F06DFD9DF8280008B185F8048026
:103030009DF8140010F0700F12D0BDF8040020802D
:10304000BDF806006080BDF80800A08046B107A961
:1030500006A800F05BF806986421484300146084D9
:103060009DF814000007CFD5BDF80C00E080BDF836
:103070000E002081BDF810006081C5E740000020EF
:10308000A40000200B49097A39B1012907D002298F
:103090000AD003290BD0002103E0FA2101E04FF40C
:1030A000FA710180002070474FF47A71F9E74FF40C
:1030B000FA61F6E7400000200C49C97A072913D2CB
:1030C000DFE801F01204060A0C0E1000BC2100E03B
:1030D00062210180002070472A21FAE71421F8E7D5
:1030E0000A21F6E70521F4E70021F2E7400000207D
:1030F000054991F8242012B14FF0FF307047C9897B
:10310000018000207047000040000020F8B51C4CF2
:1031100006460F46A07A4FF0FF3540B120686B4657
:103120000222017C60680078FFF746FB08B1284660
:10313000F8BDBDF8000040BA05B217B13846FFF738
:103140007FF86468E088FDF7DCF90746B4F9080009
:10315000FDF7CEF904462846FDF7CAF92146FDF7EA
:10316000D3F83946FDF708F90649FDF77BF8102139
:10317000FDF740F9FDF7CAF930600020F8BD000006
:103180004000002000000C4238B5724C6528A17840
:1031900062696DD026DC33286BD009DCA0F12C00ED
:1031A000072867D2DFE800F0D19AD09A9BA3B2003B
:1031B000684B38285B7874D00DDC342869D035280A
:1031C00058D100294FF0640068D0FEF7B7FC002802
:1031D00050D161A00DE3392866D061287ED182F0FC
:1031E00001007AE001256638122877D2DFE800F086
:1031F000B1670976767676767676736A63B070769E
:10320000AFAE5AA0FEF7E8F966A0FEF7E5F96BA0AD
:10321000FEF7E2F972A0FEF7DFF979A0FEF7DCF91C
:103220007EA0FEF7D9F985A0FEF7D6F98AA0FEF7B1
:10323000D3F990A0FEF7D0F998A0FEF7CDF9A0A0A1
:10324000FEF7CAF9A5A0FEF7C7F9A9A0FEF7C4F9D1
:10325000AFA0FEF7C1F9B6A0FEF7BEF9BCA0FEF71D
:10326000BBF9C3A0FEF7B8F9CAA0FEF7B5F902E0B2
:103270002BE05AE032E0D2A0FEF7AEF9D9A0FEF77B
:10328000ABF9DDA0FEF7A8F9E2A0FEF7A5F901E091
:1032900007E051E2E8A0FEF79FF900E05CE2F4A04D
:1032A000A7E283F0010001E083F002006070BDE856
:1032B000384001F0A7B8BDE8384000F043BD82F0C7
:1032C00002000AE082F0040007E082F0080004E057
:1032D00082F0100001E082F02000606138BD002023
:1032E000FEF788FC0020FEF798FCEFA081E24FF08B
:1032F0000A0029B1FEF722FC0028EFD1F0A078E205
:1033000000F0E4FF0028E9D1F2A072E24FF01400CF
:1033100029B1FEF713FC0028E0D1F3A069E200F028
:10332000D5FF0028DAD1F5A063E24FF0280029B1DB
:10333000FEF704FC0028D1D1F5A05AE200F0C6FF48
:103340000028CBD1F7A054E20EE20BE24FE241E2BB
:1033500061E20EE2A4000020444D50207365742009
:10336000746F2031303020487A2E0A003D3D3D3DBB
:103370003D3D3D3D3D3D3D3D3D3D3D3D3D3D3D209A
:1033800048454C5020434F4D4D414E4453203D3D08
:103390003D3D3D3D3D3D3D3D3D3D3D3D3D3D3D3D5D
:1033A0003D0A0000683A205072696E742048656CCE
:1033B0007020636F6D6D616E64730A00383A20533C
:1033C000657420416363656C65726F6D65746572C9
:1033D0002073656E736F72206F6E2F6F66660A00C2
:1033E000393A20536574204779726F73636F706543
:1033F0002073656E736F72206F6E2F6F66660A00A2
:10340000723A205072696E742052656769737465F0
:1034100072732076616C75650A000000613A205075
:1034200072696E7420416363656C65726F6D65745B
:10343000657220646174610A00000000673A2050E0
:1034400072696E74204779726F73636F7065206460
:103450006174610A00000000713A205072696E7454
:10346000205175617465726E696F6E20646174615C
:103470000A000000653A205072696E742045756C30
:10348000657220616E676C657320696E2064656784
:10349000726565202A203130300A0000743A2050CD
:1034A00072696E742054656D7065726174757265B1
:1034B00020696E2064656743202A203130300A007D
:1034C000703A205072696E74205065646F6D657437
:1034D000657220646174610A00000000303A205275
:1034E00065736574205065646F6D657465720A005C
:1034F000313A2053657420444D502F4D505520666D
:1035000072657175656E637920313020487A0A00E2
:10351000323A2053657420444D502F4D505520664B
:1035200072657175656E637920323020487A0A00C1
:10353000333A2053657420444D502F4D505520662A
:1035400072657175656E637920343020487A0A009F
:10355000343A2053657420444D502F4D5055206609
:1035600072657175656E637920353020487A0A007E
:10357000353A2053657420444D502F4D50552066E8
:1035800072657175656E63792031303020487A0A32
:10359000000000002C3A2053657420444D502069EF
:1035A0006E7465727275707420746F2067657374C1
:1035B000757265206576656E74206F6E6C790A0091
:1035C0002E3A2053657420444D5020696E74657204
:1035D0007275707420746F20636F6E74696E756F8E
:1035E00075730A00663A2053657420444D50206F6D
:1035F0006E2F6F66660A0000763A2053657420517C
:1036000075617465726E696F6E206F6E2F6F66667E
:103610000A000000773A2054657374206F75742097
:103620006C6F772D706F77657220616363656C20B6
:103630006D6F64650A000000733A2052756E207346
:10364000656C662D7465737420286465766963659E
:10365000206D75737420626520666163696E6720F2
:103660007570206F7220646F776E290A0000000069
:103670003D3D3D3D3D3D3D3D3D3D3D3D3D3D3D3D7A
:103680003D3D3D3D3D3D3D3D3D3D3D3D3D3D3D3D6A
:103690003D3D3D3D3D3D3D3D3D3D3D3D3D3D3D3D5A
:1036A0003D3D3D3D3D0A00005065646F6D657465AC
:1036B0007220726573657420646F6E652E0A000057
:1036C000444D502073657420746F20313020487A47
:1036D0002E0A00004D50552073657420746F203100
:1036E0003020487A2E0A0000444D50207365742023
:1036F000746F20323020487A2E0A00004D50552039
:1037000073657420746F20323020487A2E0A0000CE
:10371000444D502073657420746F20343020487AF3
:103720002E0A00004D50552073657420746F2034AC
:103730003020487A2E0A00004FF0320031B1FEF7F7
:10374000FDF900287FF4CAAD35A052E000F0BEFDBF
:103750000028F7D137A04CE000F0B8FD0028F1D1E7
:1037600039A046E0012000E00220BDE83840FEF725
:1037700017BA20780028E5D1F9B10025A5702846B0
:1037800000F0CAFC6078C10700D00825810701D588
:1037900045F07005400701D545F001052846FFF7C3
:1037A0007DFB6846FEF70AF9BDF8000000F08EFDCB
:1037B0002AA000BFFDF710FF38BDA5706846FFF7CF
:1037C00097FCBDF80000FEF7B9F9012000F0A4FC59
:1037D00026A0EFE7208B80F010002083FDF7C6FFC6
:1037E000207EC00601D425A003E02BA001E021B17A
:1037F0002FA0BDE83840FDF7EFBE142000F022F9FD
:10380000002000F0FBFC607820F0060040F0010092
:103810006070257038BDBDE8384000F043BE000040
:10382000444D502073657420746F20353020487AE1
:103830002E0A00004D50552073657420746F20359A
:103840003020487A2E0A00004D50552073657420B0
:10385000746F2031303020487A2E0A00444D5020B9
:1038600064697361626C65642E0A0000444D5020E7
:10387000656E61626C65642E0A0000004C50207118
:1038800075617465726E696F6E2064697361626CD4
:1038900065642E0A000000004C502071756174654B
:1038A000726E696F6E20656E61626C65642E0A00CF
:1038B0005761726E696E673A20466F72206C6F773F
:1038C0002D706F776572206D6F64652C20444D50AC
:1038D000206E6565647320746F206265206469736F
:1038E00061626C65642E0A007CB52D4C80208DF8D9
:1038F000000020686B460122417D60680078FEF779
:1039000095FF4FF0FF36E8BB6420FDF767FE00250A
:103910008DF8005020686B460122417D6068007878
:10392000FEF784FF70BBE574FF20A07204F8080F57
:10393000310C6070E070E1802072A0720120207173
:10394000A0761748E5766573001F257340F81A5F67
:103950004560856025776577E5834FF4FA6000F070
:1039600017FC78B9022000F035FB58B92A2000F086
:1039700077FC38B9322000F0A9FC18B90020FFF715
:103980008DFA00E004E018B9002000F057FB08B100
:1039900030467CBD002000F0D9FC00207CBD00003A
:1039A000400000202DE9FF4FDFF89480064685B0E7
:1039B00098F8250015460F464FF0FF39B0BBAFB35E
:1039C000002420E0301B102800DD102080B2834648
:1039D0003A1901469246204600F0C6FD30BB6A46C1
:1039E0005946204600F084F900BB50465A466946C5
:1039F000FCF72BFC20B16FF0010009B0BDE8F08F9F
:103A000004EB0B0084B2B442DCD3280A8DF810001A
:103A10008DF81150D8F80000444604AB417FD8F827
:103A2000040002220078FEF701FF08B14846E4E7EF
:103A3000012084F825000898E0840020DDE70000DC
:103A4000400000202DE9F84305464FF0FF392828B3
:103A500044D80727284C00267DB1012000F0CEFB7A
:103A600020208DF800004FF00108012D17D0052D02
:103A700018D88DF8018005201FE0002000F0BEFB63
:103A80008DF800608DF8017020686B460222417D40
:103A900060680078FEF7CAFE00BB267529E08DF845
:103AA0000160E8E7142D04D802208DF801000A20F7
:103AB00003E003208DF80100142000F0D1FB9DF8F5
:103AC00001006B4607EB80108DF801002068022290
:103AD000417D60680078FEF7A9FE10B14846BDE858
:103AE000F8830820A072267384F814800020FFF762
:103AF000D5F90020F3E700004000002070470000E7
:103B00002DE9FF4F814655488846002490F824103F
:103B100083B01E4625464FF0FF3BD1BB00213170DC
:103B2000817AB1B3017CA1B34A0600D502248A068A
:103B300000D5A41CCA0600D5A41C090700D5A41DE5
:103B4000016882464068097B6B4600780222FEF7D6
:103B500033FEF0B9BDF8000047BAA7427BD3DAF8CC
:103B600004205088B7EB500F14D9DAF800006B46E8
:103B7000C17C10780122FEF71FFE50B99DF80000AD
:103B8000C00607D500F0FEF86FF0010007B0BDE8F1
:103B9000F08F0DE00598FEF753FBDAF80010DAF825
:103BA00004006B46497B00782246FEF705FE08B10B
:103BB0005846EBE7B7FBF4F01099401E0870002060
:103BC0003070ECB39AF8101050460A07694613D5C6
:103BD000BDF80020062552BAA8F80020BDF8022042
:103BE00052BAA8F80220BDF8042052BAA8F804205E
:103BF000327842F008023270A5420CD0027C5206A4
:103C000009D54A19AD1C128852BAA9F80020327899
:103C100042F040023270A5420CD0027C920609D5D7
:103C20004A19AD1C128852BAA9F80220327842F023
:103C300020023270A5420ED09AF81000C00600E0B3
:103C400009E008D54819008840BAA9F8040030787E
:103C500040F010003070002098E700004000002085
:103C60002DE9F843214C0646174694F8240089466E
:103C70004FF0FF3890B3A07A80B320686B460222E1
:103C8000017B60680078FEF797FD38BBBDF8000047
:103C900045BAB54202D2002038701FE06068418802
:103CA000B5EB510F11D9216800786B46C97C012210
:103CB000FEF782FD90B99DF80000C00605D500F022
:103CC00061F86FF00100BDE8F8832068F2B24B465E
:103CD000417B60680078FEF76FFD08B14046F2E76F
:103CE000B5FBF6F0401E38700020ECE740000020E5
:103CF000F8B516000D464FF0FF371FD0104CA17AD3
:103D0000E1B1010A8DF80010C0B28DF8010041192F
:103D100060684289914211D8216800786B46C97E5B
:103D20000222FEF783FD48B92068EAB23346017EDD
:103D300060680078FEF740FD002800D03846F8BDE6
:103D40004000002038B500240D4D12E029684A7B60
:103D5000A2420CD0097EA14209D000786B46012214
:103D60002146FEF729FD10B14FF0FF3038BD641C2D
:103D7000E4B268680179A142E8D8002038BD0000AB
:103D800040000020F8B5564C4FF0FF36A07A0028CE
:103D90007DD000258DF8005020686B460122417CC3
:103DA00060680078FEF742FD002870D120686B46FD
:103DB0000122417960680078FEF738FD002866D15D
:103DC00020686B460122017960680078FEF72EFDBD
:103DD00000285CD194F82400E0B30C208DF800009A
:103DE00020686B460122017960680078FEF71EFDAD
:103DF000002872D13220FDF7F1FBC0208DF80000C1
:103E0000A07AC00702D0E0208DF8000020686B4641
:103E10000122017960680078FEF708FD00285CD176
:103E2000607C18B102208DF8000001E08DF8005090
:103E300020686B460122417C60680078FEF7F6FC42
:103E400028BB8DF8005020686B46012241796068DC
:103E500000783EE0FFE704208DF8000020686B4604
:103E60000122017960680078FEF7E0FC78B9A07C57
:103E700090B9A07AC0070FD05FF060008DF8000005
:103E800020686B46012201796068007800E024E038
:103E9000FEF7CCFC08BB01E04020EFE73220FDF745
:103EA0009DFB607C18B101208DF8000001E08DF8C9
:103EB000005020686B460122417C60680078FEF764
:103EC000B5FC50B92068064B012241796068103377
:103ED0000078FEF7ABFC002800D03046F8BD0000AB
:103EE000400000202DE9F047394C82468AB094F812
:103EF0002400894620B1002000F00EF9012600E0E0
:103F0000002607A8FFF7BEF806A8FEF7F1FF09A8EC
:103F1000FFF7D2F808A8FFF7EBF894F80A80277C9F
:103F20000025002249465046FEF700F810B16D1CEE
:103F3000022DF6DB022D1AD00025012203A96846C6
:103F4000FDF7F4FF10B16D1C022DF6DB022D0ED033
:103F500003A94846FCF7F8FFC5B269465046FEF78C
:103F6000CBFA10F0FF0F4FF0000002D002E0002566
:103F700005E001200DB940F0020040F00405FF20EB
:103F800020726072E0724FF6FF71E181A0722074BE
:103F900001202073BDF81C0000F0FAF89DF818000D
:103FA00000F018F8BDF8240000F05AF9BDF8200020
:103FB00000F08CF9404600F0C9F93846FEF76EFF74
:103FC00016B1012000F0A8F80AB02846BDE8F08735
:103FD0004000002038B5184C4FF0FF35A17A19B3D6
:103FE000022806D0042806D008280ED010281BD19D
:103FF0000DE0002000E008208DF80000607A9DF8B8
:104000000010B0EBD10F04D005E01020F4E7182029
:10401000F2E7002038BD20686B460122C179606854
:104020000078FEF703FC08B1284638BD9DF8000073
:10403000C0086072EDE7000040000020F8B5354C84
:104040000546A07CA84201D10020F8BD31484FF0C0
:10405000FF366B46D0E900104FF001020979007875
:1040600035B3FEF7A9FB70BB9DF800006B4620F04E
:1040700020008DF800002068012201796068007836
:10408000FEF7D4FBF8B90320FDF7A8FA02208DF85B
:10409000000094F8220078B382202BE020686B4661
:1040A0000122C17D60680078FEF7C0FB58B92EE0A0
:1040B000FEF782FB38B9A07AC0079DF8000003D054
:1040C00040F0200002E00CE020F020008DF800001D
:1040D00020686B460122017960680078FEF7A6FB34
:1040E00008B13046F8BD0320FDF778FA94F82200B5
:1040F00000B180208DF8000094F823000028CDD076
:104100009DF8000040F030008DF80000C6E7A5746F
:104110009AE700004000002038B51C4C94F82410A9
:1041200081421DD0002500B394F82500D0B10020B5
:1041300000F074FB0020FFF781FFE08C00F0C6F870
:104140008DF8005060686B46012200782321FEF74D
:104150006DFB012084F8240000F060FBFFF712FEE5
:10416000002038BD4FF0FF3038BD002000F056FB76
:10417000207C8DF8000060686B46012200782321C6
:10418000FEF754FB84F82450E8E7000040000020CC
:1041900038B5194C4FF0FF35A17A31B3FA2809D060
:1041A000B0F5FA7F08D0B0F57A7F0FD0B0F5FA6F8E
:1041B0001BD10DE0002000E008208DF80000207ADF
:1041C0009DF80010B0EBD10F04D005E01020F4E70B
:1041D0001820F2E7002038BD20686B460122817963
:1041E00060680078FEF722FB08B1284638BD9DF8CC
:1041F0000000C0082072EDE74000002038B5174CE1
:10420000054694F82300A84201D1002038BD0DB125
:10421000302000E000208DF80000A07C28B19DF83F
:10422000000040F002008DF8000094F8220028B150
:104230009DF8000040F080008DF8000020686B467B
:104240000122C17D60680078FEF7F0FA10B14FF0EE
:10425000FF3038BD84F82350D7E70000400000202D
:1042600038B5194C4FF0FF35A17A31B3BC2801D3D2
:10427000012010E0622801D302200CE02A2801D39B
:10428000032008E0142801D3042004E00A2801D305
:10429000052000E006208DF80000E07A9DF800106F
:1042A000884201D1002038BD20686B460122817808
:1042B00060680078FEF7BAFA08B1284638BD9DF864
:1042C0000000E072EEE7000040000020F8B51E4D4F
:1042D00004464FF0FF37A87A48B395F8240030BB66
:1042E000287D4FF47A7648B164B1282C03D8204653
:1042F000FFF7A8FB26E00020FFF7A4FB042C05D263
:10430000042406E00020FFF79DFBF9E7B44200D942
:104310003446B6FBF4F0401E8DF8000028686B466A
:104320000122417868680078FEF780FA08B13846C3
:10433000F8BD9DF80000401CB6FBF0F0E881400895
:10434000FFF78EFF0020F8BD40000020F8B50546BD
:1043500010F0700F4FF0000601D0012004E015B1FD
:104360008DF8006002E040208DF80000244C6B4680
:1043700001222068417D60680078FEF757FA4FF00F
:10438000FF3760BB9DF8000020F0400020738DF8DF
:104390000060680602D404208DF80000A80605D449
:1043A0009DF8000040F002008DF80000E80605D4FA
:1043B0009DF8000040F001008DF80000280705D4AA
:1043C0009DF8000040F038008DF8000020686B4632
:1043D0000122817D60680078FEF728FA10B1A6728C
:1043E0003846F8BD25B1082D02D00020FFF706FFA2
:1043F000A57226753220FDF7F1F80020F8BD000007
:1044000040000020F8B5124E002425467078C00701
:1044100002D008240FA000E013A0FDF7DDF87078AB
:10442000800704D544F07004357814A000E018A08B
:10443000FDF7D2F82046FFF789FF2046FEF72EFD54
:10444000002D04D0002030706846FEF751FEF8BD04
:10445000A4000020416363656C2073656E736F7206
:10446000204F6E2E0A000000416363656C20736567
:104470006E736F72204F66662E0A00004779726F66
:104480002073656E736F72204F6E2E0A000000005D
:104490004779726F2073656E736F72204F66662E58
:1044A0000A00000010B586B003A96846FFF71AFDA0
:1044B000044607280ED0E00702D107A0FDF78CF8CC
:1044C000A00702D408A0FDF787F8600702D40AA06D
:1044D000FDF782F806B010BD4779726F20666169FA
:1044E0006C65642E0A000000416363656C206661A0
:1044F000696C65642E0A0000436F6D7061737320F0
:104500006661696C65642E0A00000000072812D2FB
:10451000DFE800F0110406080A0C0E0006A008E00F
:1045200007A006E008A004E009A002E00AA000E05D
:104530000BA0FDF751B8704754617020582B200034
:1045400054617020582D200054617020592B200098
:1045500054617020592D2000546170205A2B200086
:10456000546170205A2D2000F8B516000D464FF00A
:10457000FF371FD0104CA17AE1B1010A8DF800106D
:10458000C0B28DF80100411960684289914211D88A
:10459000216800786B46C97E0222FEF747F948B9C8
:1045A0002068EAB23346017E60680078FEF73EF983
:1045B000002800D03846F8BD4000002070B5214BDF
:1045C00000252C461E68C6F30226072E14D01E684E
:1045D000C6F30226062E11D01E68C6F30226052E4B
:1045E0000FD01E68C6F30226042E0DD01B68C3F33D
:1045F0000223032B0BD00BE0042409E00125032444
:1046000006E002252C4603E00325012400E00425F2
:10461000C5F104039940C4F104040F23E34013409F
:104620000B4300F1E022190182F8001400F01F0290
:10463000012191404009800000F1E020C0F8001104
:1046400070BD00000CED00E002490843024908601B
:10465000704700000000FA050CED00E02DE9F0477E
:1046600051A688B05ACE8DE85A0050A38046D3E9AF
:104670000013CDE904134DA10020D1E90031CDE9AB
:1046800006314D4B0546024659684C4EC1F3810137
:1046900019B1012901D0022901D0314617E059682A
:1046A0005C68C1F38341C4F3C0640CB1113100E014
:1046B000891C5C68C4F300443CB1DC6A04F00F045C
:1046C000641CB6FBF4F4614301E03D4C61435C685B
:1046D000C4F303141DF8047021FA07F45F680DF1A8
:1046E000100CC7F302271CF8077024FA07F95F685B
:1046F0000DF1180CC7F3C2274FF4004A1CF80770DD
:1047000024FA07F7B8F1070F06D2DFE808F004082B
:104710000A0C0E293100084608B0BDE8F087204693
:10472000FAE74846F8E73846F6E7186BC00501D4C3
:10473000244D13E05868C0F3813030B1012806D011
:10474000022806D0032809D107E07D0806E0BD084D
:1047500004E00620B7FBF0F500E0FD082846DBE7A3
:10476000186B400602D448F21200D5E75046D3E752
:10477000186B80070ED0186B00F0030001280BD0D7
:10478000186B00F00300022808D0186BC0438007A4
:1047900006D006E03A4604E00A4602E0524600E04F
:1047A00032461046B8E7000000000000000000009C
:1047B00001020304060708090010024000127A00F3
:1047C00000093D00809FD500054901EB90110A6862
:1047D00000F01F030120984002430A607047000068
:1047E00000100240054901EB90110A6800F01F0318
:1047F0000120984082430A60704700000010024088
:10480000054901EB90110A6800F01F030120984050
:1048100002430A607047000000100240F8B5144CD3
:104820000146224694F82460D2E9000200235D1E6E
:1048300056B179B1022111E0417C10786B4601221A
:10484000FDF7F4FF68B90EE0A67A56B111B1617CAC
:1048500061B902E08DF80030EEE701218DF800101B
:10486000EAE72846F8BD9DF8000060740020F8BD16
:10487000400000202DE9F04106460F46FCF7F7F80E
:10488000041E0D4618BF0120284320F00040C0F14F
:104890007F6000F1E040C00F0ED0301C18BF012037
:1048A000384320F00040C0F17F6000F1E040C00FCD
:1048B00004BF0120FCF742FB20462946BDE8F081F9
:1048C0001048416841604168416041684160416809
:1048D0000D4A1140416041680C4A11434160016832
:1048E00041F08071016001688901FCD5416821F0C7
:1048F00003014160416841F00201416041680907DC
:10490000FCD5704700100240FFFFC2F7000004080A
:1049100070B50E484FF47A710068B0FBF1F0401E9C
:10492000B0F1807F11D24FF0E024606165170F2154
:104930002846FCF729FA0020A061072020612846BC
:10494000BDE870400021FCF71FBAFEE70000002020
:1049500002480168491C01607047000024000020E3
:10496000F0B507468FB015460E460420FCF778FEDA
:1049700000240D950C940B94CDE90964104D4FF46F
:104980004050CDE9065401260E90182209A9089638
:104990006846FBF736FC3346224629460420FCF7DE
:1049A00083FE0420FCF750FE0420FCF7B5FE042033
:1049B000FCF732FE4021384600F0DEF80FB0F0BDC3
:1049C00024440040F0B507468FB016460C464FF41D
:1049D000A060FFF7F9FE0320FCF742FE09940125D1
:1049E0000024CDE90B450D964FF440500F4E0E902C
:1049F0000A940696182209A96846CDE90745FBF7EF
:104A000000FC2B46224631460320FCF74DFE0320D6
:104A1000FCF70EFE0320FCF77FFE0320FCF7FCFDF5
:104A20008021384600F0B0F80FB0F0BD28440040B7
:104A300070B50D46044614490020611804D0B1F544
:104A4000744F04D1062000E00220FFF707FE216822
:104A50004FF6F07209040BD5400000EB5500B0FB97
:104A6000F5F000EA0201C0F3420241EA020008E068
:104A700000EB5500B0FBF5F101EA020001F00F0177
:104A80000843E06070BD000000BCFFBF2DE9F047A7
:104A9000894605462949002429488D4202D085428D
:104AA00000D1012440F21150FFF78EFE254830F866
:104AB0001400FFF789FE234E4FF09048361D012168
:104AC00056F824204046FDF7C1FB06F108070121F6
:104AD00057F824204046FDF7B9FB56F82430012250
:104AE00002214046FDF7C5FC56F824300122002182
:104AF0004046FDF7E1FC57F82430012202214046F0
:104B0000FDF7B7FC57F82430012200214046FDF79D
:104B1000D3FC284600F018F849462846FFF788FFDE
:104B20000821284600F045F80421284600F039F80D
:104B30002846BDE8F04700F02FB8000000380140DB
:104B400000440040100000200A4910B5401805D06C
:104B5000B0F5744F0CD140F20E3401E040F2114434
:104B60002046FFF74DFE2046BDE81040FFF73ABE55
:104B700010BD000000BCFFBF826822F040028260CE
:104B800082680A4382607047826822F080028260F5
:104B900082680A4382607047016841F00101016048
:104BA0007047026822F00402026002680A43026051
:104BB0007047026822F00802026002680A4302603D
:104BC000704775191A0C6A231B1C00001F20727491
:104BD000433B4138393A006B6C376F06246D6E7079
:104BE0006800000476005401F7FD00018300000016
:104BF00000080000000100183200050000002041FC
:104C00000000D242295C0F3E9A99993E3333733F9C
:104C1000295C0F3E0000700000000024000000022C
:104C20000003000000650054FFEF0000FA80000B55
:104C300012820001030C30C30E8C8CE914D54002A3
:104C400013710F8E3883F8833000F883258EF88334
:104C50003000F883FFFFFFFF0FFEA9D624000400F9
:104C60001A8279A10000003CFFFF00000010000044
:104C700038836FA2003E03304000000002CAE309FF
:104C80003E80000020000000000000004000000006
:104C900060000000000C0000000C186E000006927E
:104CA0000A16C0DFFFFF0256FD8CD377FFE1C496E2
:104CB000E0C5BEAA00000000FFFF0B2B0000165746
:104CC000000003594000000000001DFA00026C1DA6
:104CD000000000003FFFDFEB003EB3B6000D22787E
:104CE00000002F3C00000000001942B5000039A26E
:104CF0000000B365D90E9FC91DCF4C3430000000B1
:104D0000500000003BB67AE80064000000C80000D4
:104D100000000000100000001000FA921000225E57
:104D2000000D229F0001000000320000FF4600003D
:104D300063D400001000000004D6000004CC000082
:104D400004CC0000000010720000004000000000D1
:104D5000000000000006000200050007000000003F
:104D60000064000000000000000000050005006471
:104D700000200000000000000000000000004000D3
:104D80000000030000000032F8980000FF650000FA
:104D9000830F0000FF9BFC000000000000000000EB
:104DA0000000000000000000000000000000000003
:104DB00000000000000000000000000000000000F3
:104DC0000000100040000000000000060000B26A71
:104DD000000200000001FB830068000000D9FC0015
:104DE0007CF1FF830000000000650000006403E820
:104DF00000640028000000250000000016A000004C
:104E00000000100000001000002F0000000001F45E
:104E10000000100000280000FFFF4581FFFFFA722C
:104E20000000000000000000004400050005BAC6B4
:104E3000004778A20000000100000000000006000A
:104E4000000000140000254D002F706D000005AE1D
:104E5000000C02D000000000000000000000000074
:104E600000000000001B0000000000000000000027
:104E700000000000006400000008000000000000C6
:104E80000000000000000000000000000000000022
:104E90000000000000000000000000000000000012
:104EA0000000000000000000000000000000000002
:104EB00000000000000000000000000000000000F2
:104EC00000000000000000000000000000000000E2
:104ED00000000000001B00000000000000000000B7
:104EE000000E000E00000AC700040000000000329F
:104EF000FFFFFF9C00000B2B0000000200000001E0
:104F000000000064FFE50000000000000000000059
:104F1000000000000000000100000000000100008F
:104F200000000000000180000001800000018000FE
:104F3000002426D30000000000000000000600103E
:104F40000096003C0000000000000000000000008F
:104F5000000000000C0A4E68CDCF77095016675943
:104F6000C619CE8200000000000000000000000012
:104F700000000000000000000000000017D78400BF
:104F8000030000000000000000000000C7938F9D98
:104F90001E1B1C19000000000000000000000000A3
:104FA000000000000000000000000000020318855F
:104FB00000004000000000030000000300000000AB
:104FC00000000000400000000000000000000000A1
:104FD00000000000000000000000000000000000D1
:104FE00000000000000000000000000000000000C1
:104FF0000000000000000000677DDF7E72902E55EB
:105000004CF6E688000000000000000000000000F0
:1050100000000000D8DCB4B8B0D8B9ABF3F8FAB3EC
:10502000B7BB8E9EAEF132F51BF1B4B8B08097F1EC
:10503000A9DFDFDFAADFDFDFF2AAC5CDC7A90CC970
:105040002C97F1A989264666B28999A92D557DB07C
:10505000B08AA896365676F1BAA3B4B280C0B8A882
:105060009711B28398BAA3F0240844106418B2B917
:10507000B49883F1A329557DBAB5B1A38393F00009
:105080002850F5B2B6AA839328547CF1B9A3829331
:1050900061BAA2DADEDFDB819AB9AEF5606870F141
:1050A000DABAA2DFD9BAA2FAB9A38292DB31BAA2E4
:1050B000D9BAA2F8DF85A4D0C1BBAD83C2C5C7B839
:1050C000A2DFDFDFBAA0DFDFDFD8D8F1B8AAB38D67
:1050D000B4980D355DB2B6BAAF8C96198F9FA70EF6
:1050E000161EB49AB8AA872C547CBAA4B08AB6917A
:1050F000325676B28494A4C808CDD8B8B4B0F19929
:1051000082A82D557D98A80E161EA22C547C92A420
:10511000F02C5078F184A898C4CDFCD80DDBA8FC05
:105120002DF3D9BAA6F8DABAA6DED8BAB2B6869600
:10513000A6D0F3C841DAA6C8F8D8B0B4B882A8920D
:10514000F52C548898F135D9F418D8F1A2D0F8F993
:10515000A884D9C7DFF8F883C5DADF69DF83C1D84F
:10516000F40114F1A8824EA884F311D182F5D992EA
:10517000289788F109F41C1CD884A8F3C0F9D1D968
:105180009782F129F40DD8F3F9F9D1D982F4C20349
:10519000D8DEDF1AD8F1A2FAF9A88498D9C7DFF8C7
:1051A000F8F883C7DADF69DFF883C3D8F40114F1B4
:1051B00098A8822EA884F311D182F5D992509788AD
:1051C000F109F41CD884A8F3C0F8F9D1D99782F179
:1051D00049F40DD8F3F9F9D1D982F4C403D8DEDF4C
:1051E000D8F1AD8898CCA809F9D98292A8F57CF1BC
:1051F000883ACF944A6E98DB6931DAADF2DEF9D89D
:105200008795A8F221D1DAA5F9F417D9F1AE8ED09D
:10521000C0C3AE82C684C3A88595C8A588F2C0F174
:10522000F4010EF18E9EA8C63E56F554F18872F434
:105230000115F19845856EF58E9E0488F142985AC5
:105240008E9E068869F4011CF1981E1108D0F504A1
:10525000F11E970202983625DBF9D985A5F3C1DA4C
:1052600085A5F3DFD88595A8F309DAA5FAD8829247
:10527000A8F578F1881A849F26889821DAF41DF31E
:10528000D8879F39D1AFD9DFDFFBF9F40CF3D8FA17
:10529000D0F8DAF9F9D0DFD9F9D8F40BD8F3879F31
:1052A00039D1AFD9DFDFF41DF3D8FAFCA869F9F9D9
:1052B000AFD0DADEFAD9F88F9FA8F1CCF398DB45AE
:1052C000D9AFDFD0F8D8F18F9FA8CAF38809DAAF39
:1052D0008FCBF8D8F2AD978D0CD9A5DFF9BAA6F32C
:1052E000FAF412F2D8950DD1D9BAA6F3FADAA5F2EA
:1052F000C1BAA6F3DFD8F1BAB2B68696A6D0CAF381
:1053000049DAA6CBF8D8B0B4B8D8AD84F2C0DFF192
:105310008FCBC3A8B2B68696C8C1CBC3F3B0B4884E
:1053200098A821DB718D9D71859521D9ADF2FAD8B0
:105330008597A828D9F408D8F28D29DAF405D9F28E
:1053400085A4C2F2D8A88D9401D1D9F411F2D887DE
:1053500021D8F40AD8F28498A8C801D1D9F411D878
:10536000F3A4C8BBAFD0F2DEF8F8F8F8F8F8F8F814
:10537000D8F1B8F6B5B9B08A95A3DE3CA3D9F8D870
:105380005CA3D9F8D87CA3D9F8D8F8F9D1A5D9DF8E
:10539000DAFAD8B18530F7D9DED8F830ADDADED810
:1053A000F2B48C99A32D557DA083DFDFDFB591A0EA
:1053B000F629D9FBD8A0FC29D9FAD8A0D051D9F820
:1053C000D8FC51D9F9D879D9FBD8A0D0FC79D9FA31
:1053D000D8A1F9F9F9F9F9A0DADFDFDFD8A1F8F8F7
:1053E000F8F8F8ACDEF8ADDE8393AC2C547CF1A871
:1053F000DFDFDFF69D2CDAA0DFD9FADB2DF8D8A8A5
:1054000050DAA0D0DED9D0F8F8F8DB55F8D8A87873
:10541000DAA0D0DFD9D0FAF8F8F8F8DB7DF8D89C1C
:10542000A88CF530DB38D9D0DEDFA0D0DEDFD8A8FD
:1054300048DB58D9DFD0DEA0DFD0DED8A868DB702B
:10544000D9DFDFA0DFDFD8F1A888902C547C98A8A2
:10545000D05C38D1DAF2AE8CDFF9D8B087A8C1C100
:10546000B188A8C6F9F9DA36D8A8F9DA36D8A8F991
:10547000DA36D8A8F9DA36D8A8F9DA36D8F78D9D11
:10548000ADF818DAF2AEDFD8F7ADFA30D9A4DEF90C
:10549000D8F2AEDEFAF983A7D9C3C5C7F1889BA7B6
:1054A0007AADF7DEDFA4F8849408A797F300AEF294
:1054B0009819A488C6A39488F632DFF28393DB0997
:1054C000D9F2AADFD8D8AEF8F9D1DAF3A4DEA7F181
:1054D000889B7AD8F38494AE19F9DAAAF1DFD8A8B8
:1054E00081C0C3C5C7A39283F628ADDED9F8D8A37F
:1054F00050ADD9F8D8A378ADD9F8D8F8F9D1A1DA58
:10550000DEC3C5C7D8A18194F818F2B089ACC3C571
:10551000C7F1D8B8B4B09786A8319B069907AB9766
:1055200028889BF00C201440B0B4B8F0A88A9A28C0
:105530005078B79BA8295179247059446938644838
:1055400031F1BBAB88002C547CF0B38BB8A8042895
:105550005078F1B088B49726A85998BBABB38B02AA
:10556000264666B0B8F08A9CA82951798B295179D2
:105570008A2470598B2058718A4469388B39406865
:105580008A6448318B30496088F1AC002C547CF03F
:105590008CA804285078F1889726A85998AC8C02DA
:1055A000264666F0899CA8295179247059446938A7
:1055B000644831A98809205970AB11384069A8198D
:1055C0003148608CA83C415C207C00F187981986AA
:1055D000A86E767EA999882D557DD8B1B5B9A3DF7F
:1055E000DFDFAED0DFAAD0DEF2ABF8F9D9B087C4E6
:1055F000AAF1DFDFBBAFDFDFB9D8B1F1A3978E60CF
:10560000DFB084F2C8F8F9D9DED89385F14AB183C6
:10561000A308B5839A0810B79F10D8F1B0BAAEB0FE
:105620008AC2B2B68E9EF1FBD9F41DD8F9D90CF11D
:10563000D8F8F8AD61D9AEFBD8F40CF1D8F8F8ADD4
:1056400019D9AEFBDFD8F416F1D8F8AD8D61D9F4D5
:10565000F4ACF59C9C8DDF2BBAB6AEFAF8F40BD8FF
:10566000F1AED0F8AD51DAAEFAF8F1D8B9B1B6A3CF
:10567000839C08B9B1839AB5AAC0FD3083B79F1047
:10568000B58B93F20202D1ABDADED8F1B080BAABBF
:10569000C0C3B284C1C3D8B1B9F38BA391B609B466
:1056A000D9ABDEB0879CB9A3DDF1B38B8B8B8B8B31
:1056B000B087A3A3A3A3B28BB69BF2A3A3A3A3A378
:1056C000A3A3A3A3A3F1B087B59AA3F39BA3A3DCE1
:1056D000BAACDFB9A3A3A3A3A3A3A3A3A3A3A3A328
:1056E000A3A3A3A3D8D8D8BBB3B7F1AAF9DAFFD93B
:1056F000809AAA28B48098A720B79787A86688F0D0
:105700007951F1902C870CA781976293F0717160A9
:1057100085940129517990A5F1284C6C870C951836
:105720008578A38390284C6C886CD8F3A28200F211
:1057300010A8921980A2F2D926D8F188A84DD9488C
:10574000D896A83980D93CD89580A839A68698D90A
:105750002CDA87A72CD8A8899519A980D938D8A878
:105760008939A980DA3CD8A82EA83990D90CD8A8B4
:10577000953198D90CD8A809D9FFD801DAFFD89566
:1057800039A9DA26FFD890A80D8999A81080982108
:10579000DA2ED88999A83180DA2ED8A88696318059
:1057A000DA2ED8A8873180DA2ED8A88292F34180E9
:1057B000F1D92ED8A882F31980F1D92ED882ACF372
:1057C000C0A28022F1A62EA72EA92298A829DAAC81
:1057D000DEFFD8A2F22AF1A92E8292A8F23180A689
:1057E00096F1D900AC8C9C0C30ACDED0DEFFD88CAE
:1057F0009CACD010ACDE8092A2F24C82A8F1CAF22E
:1058000035F19688A6D900D8F1FF0000000000000D
:10581000555555555555C53F7D6FEB0312D6D4BF31
:105820005544880E55C1C93F3B8F68B52882A4BF37
:1058300088B20175E0EF493F09F7FD0DE13D023FF8
:105840004B2D8A1C273A03C0C88A599CE52A004080
:1058500059018D1B6C06E6BF82922EB1C5B8B33FCD
:105860004FBB610567ACDD3F182D4454FB21E93F78
:105870009BF681D20B73EF3F182D4454FB21F93F67
:10588000E2652F227F2B7A3C075C143326A6813CED
:10589000BDCBF07A8807703C075C143326A6913C98
:1058A000C4EB98999999C9BF711623FEC671BCBF04
:1058B0006D9A74AFF2B0B3BF9AFDDE522DDEADBF6C
:1058C0002F6C6A2C44B4A2BF0D5555555555D53F84
:1058D000FF8300922449C23F6E204CC5CD45B73F9F
:1058E000513DD0A0660DB13FEB0D76244B7BA93F17
:1058F00011DA22E33AAD903F000000000000000002
:105900002059000800000020700000001C0F000853
:105910009059000870000020980400002C0F000827
:1059200000A24A0400010000000000000000000086
:105930000E06110700020000040000000004000031
:10594000080000000000000000000000000000004F
:105950000000000000000000000000000000000047
:10596000C24B0008E04B00080000000000000000EF
:105970000000000000000000000000000000000027
:105980000000000000000000EC4B000800000000D8
:040000050800016985
:00000001FF
